:100000001BC035C034C033C032C031C030C02FC077
:100010002EC02DC02CC02BC02AC029C028C027C08C
:1000200026C025C024C04C696E65320048656C6CE2
:100030006F20576F726C640011241FBECFE5D4E0AF
:10004000DEBFCDBF10E0A0E6B0E0E6E1F2E002C026
:1000500005900D92A036B107D9F710E0A0E6B0E008
:1000600001C01D92A036B107E1F702D0D2C0C8CFBF
:100070009CD0B1D061E081E0B4D08CE290E082D03D
:1000800061E082E0AED086E290E07CD0FFCF853B9D
:10009000F9F0863B38F48D30E9F0803BB9F08A30D6
:1000A000D1F418C0843E51F0853E18F48F3D99F488
:1000B0000BC0863F29F08C3F29F0089581EE08950A
:1000C0008FEE089585EF089582EE08958FED0895DF
:1000D00084EE089580E008950FC000000000000045
:1000E0000000000000000000000000000000000010
:1000F0000000000000000197009779F70895CF9362
:10010000DF93EC0104C088EE93E0E6DF21972097AF
:10011000D1F7DF91CF910895939A81E090E0DCDFF1
:10012000939881E090E0D8DF089580FF02C0949A10
:1001300001C0949881FF02C0959A01C0959882FFF2
:1001400002C0969A01C0969883FF02C0979A01C098
:100150009798E2DF089582E0E8DF82E0E6DF8CE056
:10016000E4DF85E090E0CBDF08951F93182F8295A0
:100170008F70DBDF812F8F70D8DF82E390E0ACDF00
:100180001F910895CF93DF93EC0103C080DF8111AD
:10019000ECDFFE01219684918823C1F7DF91CF9196
:1001A00008959298E2DF929A08958A9A8B9A92988B
:1001B00093988C9A8D9A8E9A8F9A8FEF90E09FDF0A
:1001C000CADF929A84E1EDDF8CE0EBDF86E0E9DFC5
:1001D00082E0E7DF089581E0E4DF85E090E08FDFF3
:1001E0000895982F8150823098F4862F8150803165
:1001F00078F4913021F0923029F080E805C0862F04
:10020000815802C0862F8154CCDF82E390E064DF06
:060210000895F894FFCFF1
:00000001FF
